:100000000C9408050C944F050C944F050C944F0567
:100010000C944F050C944F050C944F050C944F0510
:100020000C944F050C944F050C94830C0C944F05C5
:100030000C942D1B0C944F050C944F050C944F05FC
:100040000C944F050C944F050C944F050C944F05E0
:100050000C944F050C94CD1B0C944F050C944F053C
:100060000C944F050C944F050C944F050C944F05C0
:100070000C944F050C944F050C944F050C944F05B0
:100080000C944F050C944F050C944F050C944F05A0
:100090000C944F050C944F050C944F050C944F0590
:1000A0000C944F050C944F050C944F05790D9B0D46
:1000B000890E9B0D890EE00D030E890E580E6B0EF6
:1000C000701170119D119D11F81134122C142C1403
:1000D0004C122C144713471302142C142C1418140C
:1000E0001F141A16041D1B062021150807091905DF
:1000F00022231C170A0B11801E352B39797B7A2C91
:100100002425180C0E0D1080742A31287C7D7F7EEA
:1001100026271213330F36802D2E302F3438378098
:10012000253032583A20253038620A000A722F638F
:100130002030313233343536370A005B735D004B83
:100140006579626F6172642073746172742E0A0043
:1001500055534220636F6E666967757265642E0A37
:10016000005B575D005B535D005B525D005B445D6F
:10017000005B435D001203480048004B0042002032
:10018000006D006F00640000000E0374002E006D0F
:10019000002E006B002E0000000403090409028DEC
:1001A00000050100A032090400000103010100095B
:1001B00021110100012240000705810308000A09FE
:1001C0000401000103010200092111010001224D77
:1001D000000705820308000A090402000103000069
:1001E00000092111010001223600070583030800E0
:1001F0000A090403000203000000092111010001A3
:1002000022220007058403200001070504032000C3
:10021000010904040001030000000921110100018B
:1002200022390007058503100001120110010000AA
:100230000008EDFEFECA04010102000105010906E5
:10024000A101050719E029E71500250195087501A9
:10025000810205081901290595057501910295018D
:100260007503910105071900297715002501957877
:1002700075018102C00631FF0974A10109751500DD
:1002800026FF009520750881020976150026FF00DB
:10029000952075089102C005010980A1018502160B
:1002A000010026B7001A01002AB7007510950181D8
:1002B00000C0050C0901A1018503160100269C025E
:1002C0001A01002A9C02751095018100C0050109E0
:1002D00002A1010901A1000509190129051500253F
:1002E00001950575018102950175038101050109DB
:1002F0003009311581257F95027508810609381569
:1003000081257F950175088106050C0A3802158143
:10031000257F950175088106C0C005010906A10168
:10032000050719E029E715002501950875018102E7
:1003300095017508810105081901290595057501C3
:1003400091029501750391010507190029FF150018
:1003500026FF00950675088100C00A002530325836
:1003600020006B6579626F6172645F7265706F7295
:10037000743A20004C45443A20253032580A006433
:10038000656C5F6B65795F6269743A2063616E27A3
:10039000742064656C3A20253032580A0061646428
:1003A0005F6B65795F6269743A2063616E277420C0
:1003B0006164643A20253032580A004F6E657368D4
:1003C0006F743A2074696D656F75740A00290A00AC
:1003D0002575002F002575005D280025640020008C
:1003E000256400200025640020002564007C002591
:1003F000303258006D6F7573656B6579205B627480
:100400006E7C782079207620685D287265702F6177
:10041000636C293A205B006D6B5F776865656C5F84
:1004200074696D655F746F5F6D6178203D20256430
:100430000A006D6B5F776865656C5F6D61785F73EF
:1004400070656564203D2025640A006D6B5F7469EA
:100450006D655F746F5F6D6178203D2025640A00D3
:100460006D6B5F6D61785F7370656564203D2025FD
:10047000640A006D6B5F696E74657276616C203D15
:100480002025640A006D6B5F64656C6179203D20F6
:1004900025640A006D6B5F776865656C5F74696DD4
:1004A000655F746F5F6D6178203D2025640A006D83
:1004B0006B5F776865656C5F6D61785F73706565AC
:1004C00064203D2025640A006D6B5F74696D655F73
:1004D000746F5F6D6178203D2025640A006D6B5F4D
:1004E0006D61785F7370656564203D2025640A0046
:1004F0006D6B5F696E74657276616C203D2025645A
:100500000A006D6B5F64656C6179203D2025640A8B
:10051000000A00257500363A20776865656C5F74BF
:10052000696D655F746F5F6D61783A20000A002520
:100530007500353A20776865656C5F6D61785F732B
:10054000706565643A20000A00257500343A20740D
:10055000696D655F746F5F6D61783A20000A0025F0
:100560007500333A206D61785F73706565643A2079
:10057000000A00257500323A20696E746572766152
:100580006C286D73293A20000A00257500313A2045
:1005900064656C6179282A31306D73293A20000A2C
:1005A000092D2056616C756573202D0A004D3E00A3
:1005B0004D25643E20003F007365742064656661CC
:1005C000756C740A00433E2000776865726520648C
:1005D000656C74613A20637572736F723D25642C8B
:1005E00020776865656C3D25640A536565206874ED
:1005F00074703A2F2F656E2E77696B697065646928
:10060000612E6F72672F77696B692F4D6F757365F8
:100610005F6B6579730A000A092D204D6F7573654C
:100620006B6579202D0A4553432F713A097175691D
:10063000740A313A0964656C6179282A31306D7326
:10064000290A323A09696E74657276616C286D7395
:10065000290A333A096D61785F73706565640A34FD
:100660003A0974696D655F746F5F6D61780A353A38
:1006700009776865656C5F6D61785F737065656447
:100680000A363A09776865656C5F74696D655F74F1
:100690006F5F6D61780A0A703A097072696E742032
:1006A00076616C7565730A643A09736574206465D4
:1006B0006661756C74730A75703A092B310A646F40
:1006C000776E3A092D310A706775703A092B31300F
:1006D0000A7067646F776E3A092D31300A0A7370B9
:1006E000656564203D2064656C7461202A206D611D
:1006F000785F7370656564202A2028726570656173
:1007000074202F2074696D655F746F5F6D61782947
:100710000A003F004D3E2000433E20004C25640A65
:10072000000A092D20436F6E736F6C65202D0A45FA
:1007300053432F713A09717569740A6D3A096D6FE7
:100740007573656B65790A000A092D204D6167692B
:1007500063202D0A643A0964656275670A783A096C
:100760006465627567206D61747269780A6B3A0915
:100770006465627567206B6579626F6172640A6D8A
:100780003A096465627567206D6F7573650A763A1C
:100790000976657273696F6E0A733A0973746174CE
:1007A00075730A633A09636F6E736F6C65206D6FC2
:1007B00064650A302D343A096C61796572302D34E4
:1007C000284631302D4634290A506175733A096242
:1007D0006F6F746C6F616465720A6E3A094E4B52AA
:1007E0004F0A003F004E4B524F3A206F66660A0098
:1007F0004E4B524F3A206F6E0A0074696D65725FFE
:1008000072656164333228293A202530346C580AE5
:10081000006B6579626F6172645F6E6B726F3A2014
:1008200025580A006B6579626F6172645F69646C58
:10083000653A2025580A006B6579626F6172645FC2
:1008400070726F746F636F6C3A2025580A00686F7E
:1008500073745F6B6579626F6172645F6C656473FA
:1008600028293A2025580A000A092D20537461745A
:100870007573202D0A004743433A20342E392E3217
:10088000204156522D4C4942433A20312E382E30C9
:1008900073766E204156525F415243483A2061764A
:1008A00072350A004F5054494F4E533A204C55462A
:1008B00041204D4F5553454B4559204558545241C1
:1008C0004B455920434F4E534F4C4520434F4D4DC0
:1008D000414E44204E4B524F204B45594D41505FA5
:1008E00053454354494F4E20343039360A0042555F
:1008F000494C443A20353166353966642D64697255
:100900007479202831363A33313A303720417567CF
:100910002033312032303136290A005649443A20FA
:1009200030784645454428742E6D2E6B2E29205074
:1009300049443A203078434146452848484B4220B4
:100940006D6F6429205645523A203078303130346A
:100950000A00444553433A20742E6D2E6B2E206BB3
:100960006579626F617264206669726D7761726524
:1009700020666F722048484B42206D6F640A000A5F
:10098000092D2056657273696F6E202D0A000A6D5D
:100990006F7573653A206F66660A000A6D6F75732E
:1009A000653A206F6E0A000A6B6579626F61726446
:1009B0003A206F66660A000A6B6579626F6172643D
:1009C0003A206F6E0A000A6D61747269783A206F7E
:1009D00066660A000A6D61747269783A206F6E0A61
:1009E000000A64656275673A206F6E0A000A6465E2
:1009F0006275673A206F66660A000A0A626F6F7452
:100A00006C6F616465722E2E2E2000433E20000024
:100A100011241FBECFEFDAE0DEBFCDBF04B603FE68
:100A200027C08091E9019091EA01A091EB01B0917A
:100A3000EC018730904BA740B04BD1F41092E90104
:100A40001092EA011092EB011092EC0114BE84B7EF
:100A5000877F84BF0FB6F894A89580916000886165
:100A600080936000109260000FBEE0E0F8E309950B
:100A700011E0A0E0B1E0E4EBF8E402C005900D92D3
:100A8000A833B107D9F721E0A8E3B1E001C01D9276
:100A9000A93EB207E1F70E94AB090C9458240C94CC
:100AA0000000FF93EF93E0913801F0913901309706
:100AB00009F00995EF91FF910895FC01859180302F
:100AC00011F0EFDFFBCF0895FF27E0E230E247FFB0
:100AD0000CC0419597FF09C0EDE260957095809537
:100AE0009095611D711D811D911D27FF02C02195EB
:100AF00030E350E2AA27660F771F881F991FAA1FAD
:100B0000A41710F0A41B63955A95A9F7AA3008F012
:100B1000A95FA05DAF93F3956115710581059105FE
:100B200041F7ED3211F4EF93F395F21718F43F9378
:100B3000F395FBCF8F91B5DFFA95E1F70895E99131
:100B4000F9918591803021F0853219F0AADFF9CF33
:100B5000089520E0E89455915532C1F3503311F4D3
:100B6000689455915A3348F4505390F3220F022E53
:100B7000220F220F200D250FF4CF0EF4219589911D
:100B80009991533619F3533729F1533559F1BC0173
:100B900088279927E8945C3621F489919991689483
:100BA0005591543639F446EF7EF077FF0DC08FEF44
:100BB0009FEF0AC055374AE039F0583540E121F03F
:100BC000523642E009F00895FF93EF937DDFEF91F5
:100BD000FF91B7CFFF93EF93FC0181918030B9F380
:100BE00060DFFBCFFF93EF9368DFF1CFDF93CF930D
:100BF000CDB7DEB72596A3DFCF91DF9108958FEFB4
:100C000084B980E485B957985F9A2E9A2F98E2E4C8
:100C1000F1E088E08E0F11928E13FDCFEAE3F1E050
:100C200088E08E0F11928E13FDCF82E491E09093B5
:100C30004D0180934C018AE391E090934B018093A6
:100C40004A0108950F931F93CF93DF9380914A0138
:100C500090914B0120914C0130914D0130934B010B
:100C600020934A0190934D0180934C01C0E0D0E065
:100C700001E010E080E090E025B1207C2C2BAC015D
:100C800033E0440F551F3A95E1F7242B25B9EAE1EB
:100C9000EA95F1F700C0E0914A01F0914B01EC0FA9
:100CA000FD1F208130E0082E02C0359527950A945B
:100CB000E2F720FD2F9AF5E3FA95F1F70000E6B58B
:100CC0002E982AE12A95F1F700C040914C015091ED
:100CD0004D01DA01AC0FBD1F4F9B0AC09801082ED1
:100CE00001C0220F0A94EAF720953C91232308C003
:100CF0006C919801082E01C0220F0A94EAF7262B66
:100D00002C9326B56E2F70E02E1718F026B530E024
:100D100004C026B530E021503F4F261B370B26304C
:100D2000310558F0E0914A01F0914B01EC0FFD1FA5
:100D30002081FA01EC0FFD1F20833AE13A95F1F78B
:100D400000C02F982E9AEBE2F1E03197F1F700C046
:100D5000000001968830910509F08ECFA0914C01DA
:100D6000B0914D01AC0FBD1FE0914A01F0914B01D4
:100D7000EC0FFD1F9C918081981751F00E946B1B16
:100D800060934E0170934F018093500190935101F5
:100D90002196C830D10509F06DCF8091E0018530F2
:100DA00021F08091E001811111C060914E0170919C
:100DB0004F0180915001909151010E94A11B61311E
:100DC00077428105910510F00E94EE1A81E0DF91D3
:100DD000CF911F910F91089520914C0130914D01B9
:100DE000F901E80FF11D808108950F931F93CF93B0
:100DF000DF938CE291E00E945D05C0E0D0E000E26C
:100E000011E0E0914C01F0914D01EC0FFD1F80814C
:100E10000E94C41A1F928F93DF93CF931F930F9357
:100E20000E94F60521960F900F900F900F900F9053
:100E30000F90C830D10529F7DF91CF911F910F9105
:100E4000089508950895569A81FF02C05E9A089504
:100E50005E9808958091650108959FB7F894109267
:100E600054019FBF9091E001943009F057C09091D8
:100E7000E9009F703091EC00232F217030FD20E8B5
:100E8000922B24E02093E9002091EB0020FF43C047
:100E90002091EE0027FF3FC020915201222321F034
:100EA0002091E80025FF37C01092520126E03091D2
:100EB000E80035FD15C03091E001343061F5309126
:100EC000EB0035FD28C0215021F481E080935201D0
:100ED00022C0EFE9FFE03197F1F700C00000E7CF53
:100EE0008093F1008091E80085FD0AC08091E800C0
:100EF00080FFFCCF8091E8008E778093E80006C0E9
:100F00008FB7F89421E0209354018FBF9F70909386
:100F1000E90080E008959F709093E9008FEF0895B5
:100F2000CF93DF9300D01F92CDB7DEB79C018091A5
:100F3000E001843019F593E099833B832A839093F1
:100F4000E9008FEF9091E800815095FD06C095ED86
:100F50009A95F1F700008111F5CF8091E80085FFA7
:100F60000DC040E050E063E070E0CE0101960E94C9
:100F7000710A8091E8008E778093E8000F900F90BF
:100F80000F90DF91CF910895CF93DF9300D01F9200
:100F9000CDB7DEB72091E001243021F522E029838E
:100FA0009B838A8383E08093E9008FEF9091E80030
:100FB000815095FD06C095ED9A95F1F700008111DD
:100FC000F5CF8091E80085FF0DC040E050E063E080
:100FD00070E0CE0101960E94710A8091E8008E7740
:100FE0008093E8000F900F900F90DF91CF910895BC
:100FF0002091E0012430F1F422E02093E9002FEF6A
:101000003091E800215035FD06C035ED3A95F1F7F5
:1010100000002111F5CF2091E80025FF0BC040E032
:1010200050E065E070E00E94710A8091E8008E77E0
:101030008093E8000895CF93DF932091E00124305E
:1010400009F048C0EC0180910A018823E1F0809109
:101050000B018823C1F085E08093E9008FEF909128
:10106000E800815095FD06C095E19A95F1F70000E2
:101070008111F5CF8091E80085FF2CC040E050E061
:1010800060E170E017C081E08093E9008FEF9091FC
:10109000E800815095FD06C095ED9A95F1F70000A6
:1010A0008111F5CF8091E80085FF14C040E050E049
:1010B00068E070E0CE010E94710A8091E8008E77AE
:1010C0008093E80080E1FE01A5E5B1E001900D927A
:1010D0008A95E1F7DF91CF91089581E791E00E9431
:1010E0005D058091DF01811109C00E94080C0E94FA
:1010F000650C8091E20084608093E20008958DE6A3
:1011000091E00E945D051092DF01089589E691E06B
:101110000C945D05209153012F5F822F62E30E94A2
:101120001E24992319F0209353010895109253011E
:1011300080915401882371F18091E001843041F560
:101140008091E9008F702091EC00922F917020FD2A
:1011500090E8892B94E09093E9009091EB0090FF48
:1011600014C09091EE0097FF10C09091E80095FF99
:1011700003C01092F100F9CF9091E80090FF05C0F4
:101180009091E8009E779093E8008F708093E9003B
:1011900010925401089542E061EC81E00E94820BBC
:1011A00042E061EC82E00E94820B42E061EC83E06D
:1011B0000E94820B42E261EC84E00E94820B42E1D9
:1011C00061EC85E00C94820B8091E201833009F49C
:1011D00055C030F4813071F0823009F48EC008952A
:1011E0008A3009F47AC08B3009F460C0893009F084
:1011F0009CC020C08091E101813A09F096C08091A5
:10120000E800877F8093E8008091E5019091E601F6
:10121000892B21F460E185E591E003C060E080E086
:1012200090E070E00E94BE0A8091E8008B77809386
:10123000E80008958091E101813209F076C0809143
:10124000E5019091E601009719F0049709F06DC04F
:101250008091E800877F8093E8008091E80082FD1C
:1012600005C08091E0018111F8CF5FC08091F1004D
:10127000809365018091E8008B7753C08091E101F4
:10128000813A09F052C08091E5019091E601892BE5
:1012900009F04BC08091E800877F8093E80080913F
:1012A000E80080FFFCCF80910A0136C08091E10107
:1012B0008132D9F58091E5019091E601892BA9F55C
:1012C0008091E800877F8093E8000E94B70B8091AF
:1012D000E30180930A010C944D148091E101813265
:1012E00021F58091E800877F8093E8000E94B70B8A
:1012F0008091E4018093660108958091E101813A33
:10130000A1F48091E800877F8093E8008091E80055
:1013100080FFFCCF809166018093F1008091E8000E
:101320008E778093E8000C94B70B08950895089584
:10133000089585E691E00E945D050C9498090E944D
:10134000EE1A8091DE01882329F00E94171B81117B
:101350000C945B0A089584B7877F84BF0FB6F89416
:10136000A895809160008861809360001092600071
:101370000FBE90E080E80FB6F894809361009093E0
:1013800061000FBE0E9496090E944E0F0E94080C39
:101390000E94650C8091E20084608093E2008DE2FF
:1013A00097E00E94BF1A78948091E001843019F090
:1013B0000E94A10EF9CF80E591E00E945D050E9498
:1013C000500F80E091E00E94BC0E8FE391E00E94FC
:1013D0005D050E9497098091E001853039F48BE327
:1013E00091E00E945D050E949F09F5CF0E94540F75
:1013F0000E94A10EF0CF0C942B1B81E691E00E947D
:101400005D050C94FB09292F332723303105C9F0E2
:1014100064F42130310581F02230310509F043C0F8
:101420008DE890E02DE931E042C021323105F1F044
:101430002232310541F137C082E190E02AE232E008
:1014400036C099278130910541F08230910541F0F5
:10145000892B49F5E9E9F1E005C0E9E8F1E002C0CE
:10146000E5E7F1E0849190E09F0121C06530D8F478
:10147000E62FF0E0EE0FFF1FED5DFE4F2081318182
:1014800089E090E014C0653070F470E0FB01EE0F6D
:10149000FF1FE75EFE4F20813181FB01EC5EFE4FB6
:1014A000808190E004C080E090E020E030E0FA012C
:1014B00031832083089580E189BD82E189BD09B42B
:1014C00000FEFDCF8091D8008F7D8093D800809161
:1014D000E00082608093E0008091E00081FDFCCF1D
:1014E0000895CF92DF92EF92FF920F931F93CF93C5
:1014F000DF93EC018B017A010E94D60B811135C07C
:10150000E114F10439F0F70180819181081B190B76
:10151000C80FD91FC12CD12C0115110529F18091BB
:10152000E80085FD18C08091E8008E778093E80080
:101530000E94A10EE114F10449F0F701808191812C
:10154000C80ED91ED182C08285E00FC00E94D60B82
:10155000882311F30AC089918093F1000150110989
:10156000FFEFCF1ADF0AD8CF80E0DF91CF911F9134
:101570000F91FF90EF90DF90CF9008952091E701B9
:101580003091E8012617370748F06115710539F4E5
:101590002091E8002E772093E80001C0B90140E0D7
:1015A00061157105A9F12091E001222309F443C0DE
:1015B000253009F442C02091E80023FD40C020916D
:1015C000E80022FD32C02091E80020FFE9CF4091E1
:1015D000F3002091F20030E0342BFC01CF016115C3
:1015E000710559F02830310540F481918093F10064
:1015F000615071092F5F3F4FF1CF41E02830310535
:1016000009F040E02091E8002E772093E800C8CF51
:101610004111C9CF0AC08091E001882361F0853073
:1016200061F08091E80083FD0AC08091E80082FFAC
:10163000F2CF80E0089582E0089583E0089581E08C
:1016400008952091E7013091E8012617370748F007
:101650006115710539F42091E8002E772093E80098
:1016600001C0B901FC0120E06115710591F1809183
:10167000E001882309F440C0853009F43FC080911F
:10168000E80083FD3DC08091E80082FD2FC080917D
:10169000E80080FFE9CF2091F3008091F20090E014
:1016A000922B6115710559F08830910540F4249111
:1016B0002093F1003196615071090196F2CF21E03B
:1016C000089709F020E08091E8008E778093E80089
:1016D000CBCF2111CCCF0AC08091E001882361F0EB
:1016E000853061F08091E80083FD0AC08091E800B8
:1016F00082FFF2CF80E0089582E0089583E00895AC
:1017000081E00895982F973058F59093E900981745
:1017100039F07091EC002091ED005091F00003C081
:10172000242F762F50E021FF19C03091EB003E7F2F
:101730003093EB003091ED003D7F3093ED00309120
:10174000EB0031603093EB007093EC002093ED00E0
:101750005093F0002091EE0027FF07C09F5FD3CF8A
:101760008F708093E90081E0089580E00895809172
:10177000E10187FF11C08091E80082FD05C08091E2
:10178000E0018111F8CF11C08091E8008B770BC088
:101790008091E001882349F08091E80080FFF8CF34
:1017A0008091E8008E778093E80008952091E4000E
:1017B0003091E50095E64091EC00842F817040FF68
:1017C00022C08091E80080FD1CC08091E001882348
:1017D00091F0853091F08091EB0085FD10C0409133
:1017E000E4005091E5004217530729F39A01915004
:1017F00011F784E0089582E0089583E0089581E080
:10180000089580E008954091E80042FFDECF0895FA
:101810000E94760C0E947E0CE0EEF0E080818160F8
:101820008083E8EDF0E080818F77808319BCA7ED9D
:10183000B0E08C918E7F8C9380818F7E808310921C
:10184000DF0108950F931F93CF93DF930E94760CCF
:101850000E947E0CC8EDD0E088818F7788838881D4
:101860008068888388818F7D888319BC1092E0010D
:101870001092DC011092DE011092DD0100EE10E00A
:10188000F80180818B7F808388818160888342E03A
:1018900060E080E00E94820BE1EEF0E080818E7FCC
:1018A0008083E2EEF0E080818160808380818860C7
:1018B0008083F80180818E7F808388818061888326
:1018C000DF91CF911F910F910895E8EDF0E08081B5
:1018D0008F7E8083E7EDF0E080818160808384E00B
:1018E00082BF81E08093DF010C94220CE8EDF0E0F0
:1018F00080818E7F80831092E20008951092DA003A
:101900001092E10008951F920F920FB60F921124CA
:101910002F933F934F935F936F937F938F939F93F7
:10192000AF93BF93EF93FF938091E10082FF0BC0D1
:101930008091E20082FF07C08091E1008B7F80935D
:10194000E1000E948A088091DA0080FF1FC0809128
:10195000D80080FF1BC08091DA008E7F8093DA0070
:101960008091D90080FF0DC080E189BD82E189BDF1
:1019700009B400FEFDCF81E08093E0010E946D0874
:1019800005C019BC1092E0010E947F088091E1001F
:1019900080FF19C08091E20080FF15C08091E200B5
:1019A0008E7F8093E2008091E20080618093E2006C
:1019B0008091D80080628093D80019BC85E0809324
:1019C000E0010E9499098091E10084FF30C080917C
:1019D000E20084FF2CC080E189BD82E189BD09B4A9
:1019E00000FEFDCF8091D8008F7D8093D80080913C
:1019F000E1008F7E8093E1008091E2008F7E8093F2
:101A0000E2008091E20081608093E2008091DC013D
:101A1000882311F084E007C08091E30087FD02C0B5
:101A200081E001C083E08093E0010E94FD09809184
:101A3000E10083FF24C08091E20083FF20C08091F9
:101A4000E100877F8093E10082E08093E0011092C3
:101A5000DC018091E1008E7F8093E1008091E200C3
:101A60008E7F8093E2008091E20080618093E200AB
:101A700042E060E080E00E94820B0E948608FF91B5
:101A8000EF91BF91AF919F918F917F916F915F91F6
:101A90004F913F912F910F900FBE0F901F9018956F
:101AA0001F93CF93DF93CDB7DEB7AA970FB6F89405
:101AB000DEBF0FBECDBFE1EEF1E088E08E0F90916A
:101AC000F10091938E13FBCF0E94E4088091E8000F
:101AD00083FF1FC18091E1019091E201492F50E005
:101AE0004A30510508F015C1FA01EA5AFF4F0C942B
:101AF0003E24803881F0823809F00BC18091E501E5
:101B00008F708093E9008091EB0085FB882780F936
:101B10001092E90006C08091DD019091DE019111E3
:101B200082609091E800977F9093E8008093F100A5
:101B30001092F100C8C0282F2D7F09F0EAC0882339
:101B400019F0823061F0E5C08091E301813009F045
:101B5000E0C0933009F080E08093DE012BC08091DB
:101B6000E301811127C08091E5018F7009F4D1C094
:101B70008093E9002091EB0020FF1CC0933021F4FA
:101B80008091EB00806214C09091EB009061909383
:101B9000EB0021E030E0A90102C0440F551F8A95F7
:101BA000E2F74093EA001092EA008091EB0088602F
:101BB0008093EB001092E9008091E800877F86C057
:101BC0008111A7C01091E3011F778091E300807815
:101BD000812B8093E3008091E800877F8093E80069
:101BE0000E94B70B8091E80080FFFCCF8091E3005A
:101BF00080688093E300111102C082E001C083E09D
:101C00008093E00186C08058823008F082C08091C5
:101C1000E3019091E4018C3D53E0950779F583E071
:101C20008A838AE289834FB7F894DE01139620E015
:101C30003EE051E2E32FF0E050935700E49120FFA3
:101C400003C0E295EF703F5FEF708E2F90E0EA30B7
:101C500010F0C79601C0C0968D939D932F5F2431DD
:101C600049F74FBF8091E800877F8093E8006AE2E0
:101C700070E0CE0101960E94BE0A14C0AE014F5F13
:101C80005F4F6091E5010E94030ABC01892B09F4B2
:101C900040C09091E800977F9093E80089819A81F5
:101CA0000E94210B8091E8008B778093E80031C07F
:101CB000803879F58091E800877F8093E8008091F3
:101CC000DC018093F1008091E8008E778093E8003A
:101CD0000E94B70B1EC081111CC09091E30192308D
:101CE000C0F48091E800877F8093E8009093DC0146
:101CF0000E94B70B8091DC01811106C08091E30046
:101D000087FD02C081E001C084E08093E0010E9471
:101D1000CB088091E80083FF0AC08091E800877FAC
:101D20008093E8008091EB0080628093EB00AA969C
:101D30000FB6F894DEBF0FBECDBFDF91CF911F91DC
:101D40000895CF938091E0018823A1F0C091E9002C
:101D5000CF709091EC00892F817090FD80E8C82BA6
:101D60001092E9008091E80083FD0E94500DCF7031
:101D7000C093E900CF91089590936C0180936B011B
:101D80000895E0916B01F0916C01309721F0019082
:101D9000F081E02D099480E00895EF92FF920F9377
:101DA0001F93CF93DF93E0916B01F0916C0130971B
:101DB000B1F18C010280F381E02D09958091CB0176
:101DC00082FF2DC080FF04C082E693E00E945D0583
:101DD000E80110E18CE5E82E83E0F82E8091CB013C
:101DE00080FF0BC088811F928F93FF92EF920E9419
:101DF000F6050F900F900F900F9011502196111132
:101E0000EDCF8091CB0180FF0AC08AE593E0DF919E
:101E1000CF911F910F91FF90EF900C945D05DF9192
:101E2000CF911F910F91FF90EF900895E0916B017A
:101E3000F0916C01309721F00480F581E02D099438
:101E400008952091690130916A018217930771F01A
:101E500090936A0180936901E0916B01F0916C01AC
:101E6000309721F00680F781E02D099408952091A4
:101E70006701309168018217930771F090936801B0
:101E800080936701E0916B01F0916C01309721F034
:101E90000084F185E02D0994089508950C944D0F68
:101EA0000E94561B0C94FF05CF92DF92EF92FF9297
:101EB0000F931F93CF93DF9300D000D000D0CDB706
:101EC000DEB70E9422068EE6C82E81E0D82E00E002
:101ED00010E0E02E802F0E94EC06F60141916F0188
:101EE000F42EF826B1F40F5F1F4F0830110589F763
:101EF0008FEF89838A831B820E945F1B8160782F0A
:101F00009D838C8349815A816B818D810E9413103E
:101F100047C09091CB0191FF04C08E830E94F506CB
:101F20008E8120E030E04F2D50E0922FBA01022E3A
:101F300002C0759567950A94E2F760FF2BC029836C
:101F4000EA8221E030E0690102C0CC0CDD1C9A95E8
:101F5000E2F790E08C219D21892B09F420E02B836E
:101F60000E945F1B8160782F9D838C8349815A81F9
:101F70006B818D810E94131049815A816B817C8114
:101F80008D810E94DB1AF801E259FE4F8081C8263C
:101F9000C08206C02F5F3F4F2830310531F6A3CFF6
:101FA0000E94DA1A0E944E1E10916D010E94C10E0D
:101FB000181741F10E94C10E80936D019091CB01E1
:101FC00092FF0EC090FF0CC01F928F9384E793E0A6
:101FD0009F938F930E94F6050F900F900F900F9094
:101FE00080916D0126960FB6F894DEBF0FBECDBF6F
:101FF000DF91CF911F910F91FF90EF90DF90CF90E5
:102000000C94EC1A26960FB6F894DEBF0FBECDBF27
:10201000DF91CF911F910F91FF90EF90DF90CF90C4
:1020200008950C942307CF93DF93CDB7DEB72B979A
:102030000FB6F894DEBF0FBECDBF942F4F83252F70
:10204000588769877A878B874A855B85452B21F07E
:102050002F3F09F59F3FF9F4DE01119686E0FD015F
:1020600011928A95E9F785E0FE01379601900D926D
:102070008A95E1F749815A816B817C818D819E81AE
:102080000E94F0162B960FB6F894DEBF0FBECDBFA0
:10209000DF91CF9108954F81588569857A858B8529
:1020A0000E94DB1AD9CFCF93882309F4A4C0C82F8C
:1020B0008CEF8C0F813A48F48C2F0E94982181116B
:1020C0009AC08C2F0E947B190CC080E28C0F883044
:1020D00058F4C77081E001C0880FCA95EAF70E94E2
:1020E000261ACF910C946A1A8BE58C0F833078F402
:1020F000C53A29F0C63A31F083E890E005C081E89E
:1021000090E002C082E890E0CF910C94210F88E526
:102110008C0F853108F06FC0C83A61F1C93A69F196
:10212000CA3A71F1CB3A79F1CC3A81F1CD3A89F1E1
:10213000CE3A91F1CF3A99F1C13BA1F1C03BA9F15F
:10214000C23BB1F1C33BB9F1C43BC1F1C53BC9F1DD
:10215000C63BD1F1C73BD9F1C83BE1F1C93BE9F13D
:10216000CA3BF1F1CB3BF9F1CC3B09F43FC080E035
:1021700090E03EC082EE90E03BC089EE90E038C037
:102180008AEE90E035C085EB90E032C086EB90E0BF
:102190002FC083EB90E02CC084EB90E029C087EB4C
:1021A00090E026C08CEC90E023C08DEC90E020C045
:1021B00083E891E01DC08AE891E01AC082E991E0CD
:1021C00017C084E991E014C081E292E011C083E27B
:1021D00092E00EC084E292E00BC085E292E008C07B
:1021E00086E292E005C087E292E002C08AE292E0D5
:1021F000CF910C94370FCF910895882329F19CEF4C
:10220000980F913A18F40E94CE190DC090E2980FE1
:10221000983058F4877091E001C0990F8A95EAF7D9
:10222000892F0E942C1A0C946A1A9BE5980F933000
:1022300020F480E090E00C94210F885A853120F43E
:1022400080E090E00C94370F0895882321F00E94DD
:10225000261A0C946A1A0895882321F00E942C1AD9
:102260000C946A1A0895CF92DF92EF92FF920F9327
:102270001F93CF93DF9300D000D000D0CDB7DEB74F
:1022800025E0FC01DE01119601900D922A95E1F7FF
:10229000FC0140813181F280258122952F7063817C
:1022A0007481672B09F4D8C23F3F19F44F3F09F4FA
:1022B000D3C26C0149833A8389819A812E830E941B
:1022C0003A19182F092F0E9439190E944918E02F36
:1022D000E295EF70F0E0E05AFF4F2E810C943E241F
:1022E000802F807F902F9F70092F882311F00295F7
:1022F000007FFF2049F0002309F45FC2802F0E9475
:10230000391A0E946A1A59C2812F0E94FD100023B7
:1023100009F4A2C2802F0E943F1A26960FB6F894A5
:10232000DEBF0FBECDBFDF91CF911F910F91FF9008
:10233000EF90DF90CF900C946A1A802F807F902FBF
:102340009F70092F803211F00295007F112319F040
:10235000113001F129C0FF20A9F0802F222349F17B
:10236000213039F526960FB6F894DEBF0FBECDBFEB
:10237000DF91CF911F910F91FF90EF90DF90CF9061
:102380000C94491A222319F0213009F465C20E94E5
:10239000521A2CC0FF20E9F0263008F05DC20E94DE
:1023A000231A802329F022C0FF20F1F0211115C04B
:1023B000802F26960FB6F894DEBF0FBECDBFDF91FB
:1023C000CF911F910F91FF90EF90DF90CF900C94E1
:1023D0002511253008F040C209C0F601858180FF33
:1023E000ECC18F708583E4CF2111FBC1802F69C1BF
:1023F000202F26952695237030E02115310521F0F8
:1024000021303105C9F028C2FF2021F0812F902F03
:10241000937002C080E090E026960FB6F894DEBF7D
:102420000FBECDBFDF91CF911F910F91FF90EF9025
:10243000DF90CF900C94210FFF2021F0812F902F5F
:10244000937002C080E090E026960FB6F894DEBF4D
:102450000FBECDBFDF91CF911F910F91FF90EF90F5
:10246000DF90CF900C94370F812FFF2019F00E943E
:10247000D41C02C00E943C1D26960FB6F894DEBF05
:102480000FBECDBFDF91CF911F910F91FF90EF90C5
:10249000DF90CF900C94C11D802F837009F078C01D
:1024A000F110DAC1812F829586958770880F880F89
:1024B000912F9F70C92ED12CE12CF12C082E04C035
:1024C000CC0CDD1CEE1CFF1C0A94D2F714FF12C0CA
:1024D0004FE050E060E070E004C0440F551F661FFD
:1024E000771F8A95D2F7CB01BA01609570958095D8
:1024F000909503C060E070E0CB01202F26952695D3
:102500002370422F50E042305105D1F04330510545
:1025100059F16C297D298E299F294130510541F1BE
:1025200026960FB6F894DEBF0FBECDBFDF91CF91D8
:102530001F910F91FF90EF90DF90CF900C945E1859
:102540006C297D298E299F2926960FB6F894DEBF27
:102550000FBECDBFDF91CF911F910F91FF90EF90F4
:10256000DF90CF900C9470180E945E18C701B601DE
:1025700026960FB6F894DEBF0FBECDBFDF91CF9188
:102580001F910F91FF90EF90DF90CF900C944C181B
:10259000FF2019F0802F817001C08695882309F4EF
:1025A0005BC1812F829586958770880F880F912F48
:1025B0009F70C92ED12CE12CF12C082E04C0CC0C1C
:1025C000DD1CEE1CFF1C0A94D2F714FF12C04FE072
:1025D00050E060E070E004C0440F551F661F771F95
:1025E0008A95D2F7CB01BA01609570958095909548
:1025F00003C060E070E0CB01202F26952695237064
:10260000422F50E042305105D1F04330510559F18D
:102610006C297D298E299F294130510541F126964B
:102620000FB6F894DEBF0FBECDBFDF91CF911F91E3
:102630000F91FF90EF90DF90CF900C9415196C29BB
:102640007D298E299F2926960FB6F894DEBF0FBEEE
:10265000CDBFDF91CF911F910F91FF90EF90DF9051
:10266000CF900C9427190E941519C701B601269620
:102670000FB6F894DEBF0FBECDBFDF91CF911F9193
:102680000F91FF90EF90DF90CF900C940319103FC3
:1026900041F118F4103E48F48BC0123F09F450C0C9
:1026A000D8F1133F09F460C083C01F70802F8F7171
:1026B000FF2021F00E949C18812F7BCE0E94BD1824
:1026C000812F26960FB6F894DEBF0FBECDBFDF91E7
:1026D000CF911F910F91FF90EF90DF90CF900C94CE
:1026E0002C11FF20A9F0253008F0B6C0802F8F7183
:1026F00026960FB6F894DEBF0FBECDBFDF91CF9107
:102700001F910F91FF90EF90DF90CF900C94E21803
:10271000263008F0A1C0EACFFF20A1F0802F8F71F2
:1027200026960FB6F894DEBF0FBECDBFDF91CF91D6
:102730001F910F91FF90EF90DF90CF900C949C1819
:10274000FF2061F3802F8F7126960FB6F894DEBFBD
:102750000FBECDBFDF91CF911F910F91FF90EF90F2
:10276000DF90CF900C94BD18FF2091F0802F8F71D7
:1027700026960FB6F894DEBF0FBECDBFDF91CF9186
:102780001F910F91FF90EF90DF90CF900C948718DE
:1027900026960FB6F894DEBF0FBECDBFDF91CF9166
:1027A0001F910F91FF90EF90DF90CF900C948218C3
:1027B000FF20A1F0222309F4B1CF812F26960FB676
:1027C000F894DEBF0FBECDBFDF91CF911F910F9167
:1027D000FF90EF90DF90CF900C945310222309F4D8
:1027E000B1CF812F26960FB6F894DEBF0FBECDBFB6
:1027F000DF91CF911F910F91FF90EF90DF90CF90DD
:102800000C94FD10402F4F70612FC6010E944E1C8A
:1028100026960FB6F894DEBF0FBECDBFDF91CF91E5
:102820001F910F91FF90EF90DF90CF900C94941731
:10283000402F4F70612FC60126960FB6F894DEBF69
:102840000FBECDBFDF91CF911F910F91FF90EF9001
:10285000DF90CF900C94511C26960FB6F894DEBFF3
:102860000FBECDBFDF91CF911F910F91FF90EF90E1
:10287000DF90CF9008950E94461A0E94151A0E9478
:102880006A1A0E94F31E0E94C11D80E090E00E941F
:10289000210F80E090E00C94370F0E94361A0C94C0
:1028A0003B140E943A19292F22952F7030E02C30CA
:1028B00031054CF42A3031056CF4225031092230B4
:1028C000310588F407C02C30310549F02F3031052F
:1028D00031F009C0803E48F0803F29F406C093FBE8
:1028E000882780F9089580E0089581E00895CF93C6
:1028F000DF9300D000D01F92CDB7DEB70F900F90BE
:102900000F900F900F90DF91CF910895CF93DF93A9
:1029100000D000D000D0CDB7DEB726960FB6F89421
:10292000DEBF0FBECDBFDF91CF9108951F93CF9330
:10293000DF93C091760116E080917701C81799F076
:10294000D0E01C9FF0011D9FF00D1124E858FE4FB0
:102950004081518162817381848195810E948614B6
:102960002196C770E9CFDF91CF911F9108954091D3
:10297000A8015091A9016091AA017091AB018091C9
:10298000AC019091AD010C9486148091AD018295BB
:102990008F7009F054C08091AA01882309F44FC0B8
:1029A00080917601A09177016091A8017091A901B1
:1029B0004091AB015091AC01B6E08A1709F43FC0D9
:1029C00090E041155105C1F17F3F11F46F3FA1F136
:1029D000B89FF001B99FF00D1124E858FE4F2181F6
:1029E00072132AC02081621327C02281211124C0C2
:1029F000238134812417350710F421503109241B19
:102A0000350B2C323140C0F42091AD012F70206184
:102A10002093AD0126E0289FF001299FF00D11249D
:102A2000E358FE4F80818F708061808388EA91E057
:102A30000E9433110C94961401968770BECF0895AE
:102A4000CF92DF92EF92FF920F931F93CF93DF937A
:102A5000CDB7DEB762970FB6F894DEBF0FBECDBF1D
:102A60008C0185E0F801DE011D9601900D928A959A
:102A7000E1F7D8014C9111965C91119712966C91E7
:102A800012971396CD90DC9014973091A801709115
:102A9000A9018091AB019091AC01009709F473C139
:102AA0007F3F19F43F3F09F46EC1E090AA01EE2088
:102AB00009F4C5C02091AD01C816D90650F0F60141
:102AC000E81BF90BCF01FF24F3948C329140C8F03E
:102AD00009C0809590958C0D9D1DFF24F3948C3238
:102AE000914078F0F12C207F09F0C6C07C2DD98A66
:102AF000C88A89890E94771488EA91E00E9433117C
:102B0000B1C0822F807F09F045C0751313C0341304
:102B100011C061110FC02F7020612093AD010E9480
:102B2000B71488EA91E00E9433118091AD01F80159
:102B300085832EC0CD2819F15F3F11F44F3FF9F086
:102B4000F62E61111CC0809176012091770136E04C
:102B5000821709F45BC090E0389FF001399FF00DB7
:102B60001124E858FE4F7181571306C07081471336
:102B700003C07281711103C001968770E9CFF62EF0
:102B8000662309F41DC18091AD0181608093AD0180
:102B9000F12C16C1751309C0341307C0611105C0AB
:102BA0008091AD01F8018583C8C04D875E878D8512
:102BB0009E856A8B0E9451146A898823E1F16623FD
:102BC000D1F12091AD01822F82958F7090E0029714
:102BD00074F08091A8019091A90198878F8319863C
:102BE000DB86CA862C87CE0107960E94331186E0C9
:102BF000F801A8EAB1E001900D928A95E1F70E94F0
:102C0000C5140E94B714FF24F394DAC04D875E8781
:102C10008D859E850E943A19292F22952F7030E0CC
:102C2000223031050CF0BFC09F7009F0B9C0805E42
:102C3000883008F4C5C0C8010E943311E4CFC8161B
:102C4000D90608F453C0F601E81BF90BCF018C320A
:102C5000914008F453C0F12C7C2DD98AC88A898907
:102C60000E947714E8EAF1E086E0DF011D928A9580
:102C7000E9F70E94B714A4C0751314C0341312C02E
:102C8000611110C08091AD01F8018583C8010E94D7
:102C9000331186E0E8EAF1E0DF011D928A95E9F759
:102CA000FE2C8EC04D875E878D859E856A8B0E9427
:102CB00051146A89882309F4BECF662309F4BBCF77
:102CC0002091AD01822F82958F7090E002970CF4D5
:102CD0008ECF8091A8019091A9019A8389831B824C
:102CE000DD82CC822E83CE0101967FCF8095909598
:102CF0008C0D9D1D8C32914008F0ADCFF62E6623D1
:102D000009F499CF75132EC034132CC02091AD0156
:102D100020FD1FC0822F82958F70D9F0D8011596A3
:102D20002C9315978F3049F08F5F982F9295907F55
:102D3000822F8F70892B15968C93C8010E943311B6
:102D400086E0F801A8EAB1E001900D928A95E1F7DA
:102D500090CF86E0F801A8EAB1E001900D928A9543
:102D6000E1F72EC04D875E878D859E850E945114A8
:102D700081113DCF8091AD0181608093AD01C8018B
:102D80000E9433111DC0662309F455CF4D875E871D
:102D90008D859E850E945114882309F44CCF27CF3E
:102DA000811145CF0DC0243031050CF044CF9F7008
:102DB00009F43DCFD80115969C91907F09F037CF4B
:102DC0008F2D62960FB6F894DEBF0FBECDBFDF9198
:102DD000CF911F910F91FF90EF90DF90CF900895CA
:102DE0001F93CF93DF93CDB7DEB72C970FB6F89430
:102DF000DEBF0FBECDBF4F83588769877A878B8729
:102E00009C87CE0107960E942015882369F08F8148
:102E100098852A853B85232BF1F19F3F09F063C0FC
:102E20008F3F09F060C037C086E0FE013796DE01B3
:102E3000119601900D928A95E1F76F817885EA8568
:102E4000FB85309741F17F3F11F46F3F21F12091D5
:102E5000770130E0C901019687709927409176018A
:102E600050E08417950709F447C069837A83FD838E
:102E7000EC8396E0929FD001939FB00D1124A85847
:102E8000BE4FFE01319601900D929A95E1F7809325
:102E900077010E94961416E0809176019091770157
:102EA0008917C1F1189FC001112488589E4F0E94B4
:102EB0002015882379F1E09176011E9FF0011124FD
:102EC000E858FE4F408151816281738184819581F0
:102ED0000E9486148091760190E001968770992770
:102EE00080937601D9CF4F81588569857A858B8506
:102EF0009C850E948614CFCF0E944D1410927701BA
:102F000010927601E8EAF1E086E0DF011D928A95F1
:102F1000E9F7C1CF2C960FB6F894DEBF0FBECDBF38
:102F2000DF91CF911F910895DF92EF92FF920F935F
:102F30001F93CF93DF93FC01892B09F48AC0E12C06
:102F4000F12CDD24D394EF0121968491853709F487
:102F500061C058F4843708F04EC0843008F06AC06D
:102F60008130D1F0823071F174C0883709F45DC0CE
:102F700050F4863709F455C0873709F06AC08E2DA2
:102F80000E94331A54C09CE7980F903708F061C034
:102F90008F770E94FD1050C08F010E5F1F4FFE0102
:102FA000849190E2980F983050F48770FD2D01C005
:102FB000FF0F8A95EAF78F2F0E94391A14C00E94DA
:102FC000531013C08F010E5F1F4FFE01C49180E2AA
:102FD0008C0F883060F4C7708D2D01C0880FCA95A2
:102FE000EAF70E943F1A0E946A1AE80125C08C2F56
:102FF0000E94FD10FACF9F012E5F3F4FFE01C4914A
:10300000CC2369F08FE99FE00197F1F700C0000041
:10301000C150F6CF9F012E5F3F4FFE01F490E901B2
:103020000BC00E94231AE82E07C00E94361A0E9485
:103030006A1A02C00E9453108F2D882341F0EFE9D5
:10304000FFE03197F1F700C000008150F6CFFE019C
:103050007ACFDF91CF911F910F91FF90EF90DF908A
:1030600008956093B2017093B3018093B40190937B
:10307000B5010E94EA1A0C943B146093AE01709360
:10308000AF018093B0019093B1010E94EB1A0C94B0
:103090003B1408950C9431180F931F930091B201C3
:1030A0001091B3012091B4013091B501602B712BC7
:1030B000822B932B1F910F910C9431180F931F9318
:1030C0000091B2011091B3012091B4013091B5018A
:1030D00060237123822393231F910F910C94311845
:1030E0000F931F930091B2011091B3012091B4018D
:1030F0003091B50160277127822793271F910F9187
:103100000C94311860E070E0CB010C943D180F93E3
:103110001F9341E050E060E070E08A019B0104C031
:10312000000F111F221F331F8A95D2F7C901B80162
:103130001F910F910C943D180F931F9341E050E0A5
:1031400060E070E004C0440F551F661F771F8A952A
:10315000D2F78091AE019091AF01A091B001B091F2
:10316000B1018A019B01082B192B2A2B3B2BC9018A
:10317000B8011F910F910C943D180F931F9341E0DC
:1031800050E060E070E004C0440F551F661F771FD9
:103190008A95D2F740955095609570958091AE01D3
:1031A0009091AF01A091B001B091B1018A019B0152
:1031B000082319232A233B23C901B8011F910F912A
:1031C0000C943D180F931F9341E050E060E070E0D5
:1031D00004C0440F551F661F771F8A95D2F7809150
:1031E000AE019091AF01A091B001B091B1018A01FF
:1031F0009B01082719272A273B27C901B8011F91DE
:103200000F910C943D180F931F930091AE011091F4
:10321000AF012091B0013091B101602B712B822B55
:10322000932B1F910F910C943D180F931F930091B6
:10323000AE011091AF012091B0013091B101602336
:103240007123822393231F910F910C943D180F93A8
:103250001F930091AE011091AF012091B001309108
:10326000B10160277127822793271F910F910C943A
:103270003D180895CF92DF92EF92FF920F931F9324
:10328000CF93DF938C01C090B201D090B301E09056
:10329000B401F090B5014091AE015091AF01609141
:1032A000B0017091B101C42AD52AE62AF72ACFE1EC
:1032B000D0E0D701C6010C2E04C0B695A79597950E
:1032C00087950A94D2F780FF07C0B8018C2F0E941F
:1032D000231C8130910531F4219758F7B80180E023
:1032E0000E94231CDF91CF911F910F91FF90EF90CF
:1032F000DF90CF90089590910A01992321F0909149
:103300000B01911109C020910C0130910D01F901BF
:1033100032969FEF40E030C0982F969596959695FF
:103320009F30A0F4E0910C01F0910D01E90FF11D27
:10333000877021E030E0A90102C0440F551F8A9533
:10334000E2F7CA019181892B818308959091CB0185
:1033500090FF23C01F928F938DE993E09F938F93EB
:103360000E94F6050F900F900F900F9008959F3FC9
:1033700039F04F5F4E3041F051915813F8CF0DC0E6
:103380005111F7CF942FF5CF9F3F39F0F901E90F95
:10339000F11D97FDFA9582830895089590910A0191
:1033A000992321F090910B01911109C020910C01FA
:1033B00030910D01F9013296205F3F4F30C0982FB8
:1033C0009695969596959F30A8F4E0910C01F09112
:1033D0000D01E90FF11D877021E030E0A90102C065
:1033E000440F551F8A95E2F7CA0180959181892380
:1033F000818308959091CB0190FF16C01F928F9307
:103400008FE793E09F938F930E94F6050F900F90A4
:103410000F900F9008953196E217F30729F09081ED
:103420009813F9CF1082F7CF089581E090E0E091F2
:103430000C01F0910D01E80FF91F10820196803107
:103440009105A9F708958091CA0108959091CA0144
:10345000892B8093CA01089580959091CA01892390
:103460008093CA0108958093CA0108951092CA01F9
:1034700008959091C901892B8093C9010895809581
:103480009091C90189238093C90108951092C901BF
:1034900008958093B8010E945F1B9093B7018093B9
:1034A000B60108951092B8011092B7011092B601BA
:1034B000089580910C0190910D01FC0131969C01C1
:1034C000205F3F4F80E0919191118F5FE217F307EA
:1034D000D1F70895E0910C01F0910D018091CA019E
:1034E0008083E0910C01F0910D0190818091C901E0
:1034F000892B80838091B8018823D9F10E945F1BBA
:103500002091B6013091B7018217930748F00E94CD
:103510005F1B2091B6013091B701821B930B0AC04B
:103520000E945F1B2091B6013091B7012095309524
:10353000820F931F8C32914070F08091CB0180FFFD
:1035400008C08BEB93E09F938F930E94F6050F903A
:103550000F900E94521AE0910C01F0910D019081A0
:103560008091B801892B80830E94591A81110E9491
:10357000521A80910C0190910D010C94CD0E9093F4
:1035800039018093380108958295982F9C7C392FBA
:1035900036953695282F237344E0249FC0011124CB
:1035A000932F982B292F2A7A2695892F8575880F96
:1035B000822B08950895CF93DF9300D000D01F92FF
:1035C000CDB7DEB70F900F900F900F900F90DF9157
:1035D000CF910895089508950C9411108091E00101
:1035E000843021F11092CC0120E488E190E00FB604
:1035F000F894A895809360000FBE2093600083B775
:10360000817F846083BF83B7816083BF789488950E
:1036100083B78E7F83BF0FB6F894A8958091600022
:10362000886180936000109260000FBE0895CF9370
:103630000E9421070E9422060E942207C0E08C2FD0
:103640000E94EC06811104C0CF5FC830C1F701C0F1
:1036500081E0CF9108950C944D141F920F920FB6F4
:103660000F9211248F939F93AF93BF938091CC01BE
:10367000811113C08091CD019091CE01A091CF0115
:10368000B091D0014196A11DB11D8093CD019093C1
:10369000CE01A093CF01B093D001BF91AF919F9184
:1036A0008F910F900FBE0F901F90189582E084BDF0
:1036B00093E095BD9AEF97BD80936E0008952FB764
:1036C000F8948091CD019091CE01A091CF01B0915D
:1036D000D0012FBF08952FB7F8946091CD0170915C
:1036E000CE018091CF019091D0012FBF0895CF924C
:1036F000DF92EF92FF920F931F932FB7F8944091B0
:10370000CD015091CE016091CF017091D0012FBFBA
:103710006A017B01EE24FF248C0120E030E0C0161A
:10372000D106E206F30610F4415051099A01281B14
:10373000390BC9011F910F91FF90EF90DF90CF904F
:103740000895CF92DF92EF92FF920F931F932FB7BE
:10375000F894C090CD01D090CE01E090CF01F090D0
:10376000D0012FBF97018601061B170B280B390BC1
:10377000C616D706E806F90618F0C901B80106C052
:10378000C901B80161507109810991091F910F9117
:10379000FF90EF90DF90CF9008951F920F920FB699
:1037A0000F9211248F939F93AF93BF938091CD017C
:1037B0009091CE01A091CF01B091D0010196A11DB1
:1037C000B11D8093CD019093CE01A093CF01B09312
:1037D000D001BF91AF919F918F910F900FBE0F902D
:1037E0001F9018950E94080CF8942FEF87EA91E635
:1037F000215080409040E1F700C0000087E090EB4E
:10380000DC018093E9019093EA01A093EB01B0936E
:10381000EC019CE088E10FB6F894A89580936000D5
:103820000FBE90936000FFCF28E0929FF00111241B
:10383000E80FF11DE052FF4F8491982F90778F7021
:1038400092959F700895CF93C82FCB010E94141CAE
:10385000292F30E0E82FF0E0A90164E0440F551F64
:103860006A95E1F74E2B5F2B4038510519F480E043
:1038700090E012C088E0C89F200D311D112484E023
:10388000220F331F8A95E1F7E20FF31FEE0FFF1FA0
:10389000E050F84985919491CF91089580E090E0AF
:1038A000089508958091D30180FF0BC060911101AC
:1038B00085E0689FB00111247595679575956795AA
:1038C0002BC081FF09C06091110185E0689FB001A4
:1038D00011247595679520C082FF07C06091110182
:1038E00085E0689FB001112417C09091D4019923FD
:1038F000D1F060911001961788F72091110185E0B1
:10390000289F90011124929FA001939F500D112494
:1039100070E0CA010E942A246038710540F46115E4
:10392000710539F002C065E070E0862F08958FE7D9
:10393000089581E008958091D30180FF08C06091CF
:103940000F0170E0759567957595679521C081FFAA
:1039500006C060910F0170E07595679519C082FFF0
:1039600004C060910F0170E010C09091D4019923C0
:10397000C1F060910E019617A0F780910F01899F09
:10398000C001112470E00E942A246038710528F4D7
:103990006115710521F0862F08958FE7089581E064
:1039A000089561E070E0F4CF803F21F40E94521C42
:1039B000819504C0813F29F40E94521C8093D70155
:1039C0000895823F21F40E94521C819504C0833FD8
:1039D00029F40E94521C8093D6010895893F19F45E
:1039E0000E949B1C05C08A3F31F40E949B1C81955C
:1039F0008093D80108958B3F21F40E949B1C8195F0
:103A000004C08C3F29F40E949B1C8093D901089527
:103A1000843F21F48091D501816017C0853F21F456
:103A20008091D501826011C0863F21F48091D5013B
:103A300084600BC0873F21F48091D501886005C068
:103A4000883F31F48091D50180618093D50108953C
:103A50008D3F21F48091D30181600BC08E3F21F412
:103A60008091D301826005C08F3F29F48091D301FA
:103A700084608093D3010895803F39F48091D70109
:103A800087FF6CC01092D70169C0813F29F48091F3
:103A9000D7011816BCF362C09091D601823F29F479
:103AA00097FF5CC01092D60159C0833F19F41916D4
:103AB000CCF354C0893F41F48091D80118160CF022
:103AC0004DC01092D8014AC08A3F29F48091D80194
:103AD00087FF44C0F6CF8B3F39F48091D90187FF2F
:103AE0003DC01092D9013AC08C3F29F48091D90190
:103AF0001816BCF333C0843F21F48091D5018E7F2A
:103B000017C0853F21F48091D5018D7F11C0863F7C
:103B100021F48091D5018B7F0BC0873F21F48091E8
:103B2000D501877F05C0883F31F48091D5018F7E14
:103B30008093D50113C08D3F21F48091D3018E7FF6
:103B40000BC08E3F21F48091D3018D7F05C08F3F44
:103B500029F48091D3018B7F8093D3018091D6018A
:103B600081110EC08091D70181110AC08091D801C6
:103B7000811106C08091D901811102C01092D40137
:103B800008958091CB0183FF7EC084EF93E00E9473
:103B90005D058091D5011F928F938FEE93E09F93E7
:103BA0008F930E94F6058DEE93E00E945D05809153
:103BB000D601282F082E000C330B3F938F938AEEEB
:103BC00093E09F938F930E94F60588EE93E00E9406
:103BD0005D058091D701282F082E000C330B3F93F1
:103BE0008F9385EE93E09F938F930E94F60583EE6B
:103BF00093E00E945D058091D801282F082E000CCB
:103C0000330B3F938F9380EE93E09F938F930E94AB
:103C1000F6058EED93E00E945D058091D901282F75
:103C2000082E000C330B3F938F938BED93E09F9303
:103C30008F930E94F60588ED93E00E945D058091C8
:103C4000D4011F928F9385ED93E09F938F930E94F1
:103C5000F60583ED93E00E945D058091D3011F92EC
:103C60008F9380ED93E09F938F930E94F6058DECE8
:103C700093E00E945D058DB79EB74C960FB6F89401
:103C80009EBF0FBE8DBF85ED91E00E94160F0E9472
:103C90005F1B9093D2018093D10108951F93CF931E
:103CA000DF938091D1019091D2010E94771BAC01EA
:103CB0009091D401992321F02091120130E006C0A7
:103CC000209113018AE0289F900111244217530785
:103CD00008F485C08091D601C091D701D091D80158
:103CE0001091D901811107C0C11175C0D11173C0E4
:103CF000111171C074C09F3F19F09F5F9093D40160
:103D0000181624F40E94521C8093D6018091D6018B
:103D100087FF05C00E94521C81958093D6011C1616
:103D200024F40E94521C8093D7018091D70187FF11
:103D300005C00E94521C81958093D7016091D601E5
:103D4000662331F1C091D701CC2311F1062E000C6E
:103D5000770B880B990B0E94252323E333E343E37E
:103D60005FE30E9489230E94ED226093D6016C2FAD
:103D7000CC0F770B880B990B0E94252323E333E3A9
:103D800043E35FE30E9489230E94ED226093D70101
:103D90001D1624F40E949B1C8093D8018091D801A9
:103DA00087FF05C00E949B1C81958093D801111646
:103DB00024F40E949B1C8093D9018091D90187FF34
:103DC00005C00E949B1C81958093D901DF91CF9102
:103DD0001F910C94C11D9F3F09F08FCF97CFDF91AA
:103DE000CF911F910895E5EDF1E085E0DF011D928F
:103DF0008A95E9F71092D4011092D301089587E1D2
:103E000096E00E945D051F9281E08F931F9285E0EE
:103E10008F9389EC95E09F938F930E94F6050F9006
:103E20000F900F900F900F900F9008958330E9F14D
:103E300028F4813061F0823009F10895853009F469
:103E400062C008F449C0863009F474C008958091B6
:103E50001301262F30E0280F311D2F3F310524F4A8
:103E6000680F6093130103C08FEF8093130180915B
:103E700013011F928F9382E095E072C0809112012E
:103E8000262F30E0280F311D2F3F310524F4680F15
:103E90006093120103C08FEF809312018091120191
:103EA0001F928F9380EF94E05BC080911101262FC9
:103EB00030E0280F311D2F3F310524F4680F609347
:103EC000110103C08FEF80931101809111011F92A6
:103ED0008F938DED94E044C080911001262F30E047
:103EE000280F311D2F3F310524F4680F6093100116
:103EF00003C08FEF80931001809110011F928F9368
:103F000088EC94E02DC080910F01262F30E0280F1F
:103F1000311D2F3F310524F4680F60930F0103C05A
:103F20008FEF80930F0180910F011F928F938FEA83
:103F300094E016C080910E01262F30E0280F311D2D
:103F40002F3F310524F4680F60930E0103C08FEFFB
:103F500080930E0180910E011F928F9384E994E06B
:103F60009F938F930E94F6050F900F900F900F90E4
:103F70000895833081F128F4813059F08230D1F0F6
:103F80000895853009F449C0B8F1863009F456C067
:103F9000089580911301681720F4861B8093130104
:103FA00002C010921301809113011F928F9385E834
:103FB00094E054C080911201681720F4861B80930E
:103FC000120102C010921201809112011F928F9370
:103FD00083E794E043C080911101681720F4861BA9
:103FE0008093110102C010921101809111011F9262
:103FF0008F9380E694E032C080911001681720F41E
:10400000861B8093100102C0109210018091100154
:104010001F928F938BE494E021C080910F01681769
:1040200020F4861B80930F0102C010920F01809133
:104030000F011F928F9382E394E010C080910E01D4
:10404000681720F4861B80930E0102C010920E01A7
:1040500080910E011F928F9387E194E09F938F933D
:104060000E94F6050F900F900F900F900895CF9338
:10407000C82F1F928F938CE197E09F938F930E949C
:10408000F60581E090E0A0E0B0E0BC01CD0104C005
:10409000660F771F881F991FCA95D2F70E944A188A
:1040A0000F900F900F900F90CF910C944D14CF93D1
:1040B0008732A8F58E3108F02BC1803109F49FC0FA
:1040C000F8F4873009F464C0A8F4863009F024C1FC
:1040D0008091CB01817F8E7F8093CB0181E297E03D
:1040E0000E945D058BE09AE00E945D0581E080936F
:1040F000DB014CC08B30F1F18E3009F46CC00CC187
:10410000863109F4B0C020F4813109F4EDC004C156
:10411000893109F491C08B3109F449C0FDC088335D
:1041200049F150F4893209F4F1C0853309F4EEC045
:10413000873209F0F1C0EAC0833409F4E7C028F4FB
:104140008A3308F4E9C08953E4C0883409F0E4C034
:104150000E944D148AEF99E00E945D052FEF83EDD8
:1041600090E3215080409040E1F700C000000E94A1
:10417000F21B0CC088E497E05CC081EE99E00E94DD
:104180005D058091CB0181608093CB01C1E0C9C006
:104190008091CB01C82FC17080FFEFCF8DEE99E0E9
:1041A0000E945D058091CB01817F8E7F3DC0909103
:1041B000CB0191FBCC27C0F981E0C827892FC0FB38
:1041C00081F98093CB01CC2319F084ED99E027C0CD
:1041D00086EC99E02EC09091CB0192FBCC27C0F9E0
:1041E00081E0C827892FC0FB82F98093CB01CC23C3
:1041F00019F087EB99E013C087EA99E01AC0909113
:10420000CB0193FBCC27C0F981E0C827892FC0FBE5
:1042100083F98093CB01CC2351F08BE999E00E9484
:104220005D058091CB0181608093CB017AC08EE8DF
:1042300099E00E945D05AACF8FE799E00E945D0595
:1042400082E599E00E945D058BE199E00E945D05A1
:104250008EEE98E00E945D0584EA98E00E945D057C
:1042600086E798E0E6CF88E698E00E945D050E9428
:10427000C10E1F928F938EE498E09F938F930E94BC
:10428000F60580910A011F928F9387E398E09F9330
:104290008F930E94F605809166011F928F9384E2AE
:1042A00098E09F938F930E94F60580910B011F92D7
:1042B0008F9381E198E09F938F930E94F6050E946F
:1042C0006B1B9F938F937F936F938AEF97E09F93DE
:1042D0008F930E94F6058DB79EB746960FB6F89459
:1042E0009EBF0FBE8DBF52CF0E944D14C0910B01D7
:1042F00081E0C827C0930B01CC2329F080EF97E021
:104300000E945D050EC085EE97E093CF80E001C06E
:104310008D510E9437203ACF83EE97E00E945D05D1
:10432000C0E08C2FCF91089580E0089580E008953B
:10433000CF93C82F8091DB01813071F020F0823063
:1043400009F44BC042C1E0910C01F0910D01808154
:10435000823209F03CC107C0E0910C01F0910D01DF
:104360008081823261F48C2F0E949421811104C0DB
:104370008C2F0E9457202FC081E090E02CC08C2F02
:104380000E949621811126C0C431E1F070F4CB3037
:1043900081F0C031D1F40E94FF1E84E197E00E94B9
:1043A0005D0582E08093DB0115C0C93259F0C83346
:1043B00061F481E297E00E945D0588E197E00E9448
:1043C0005D0508C01092DB0104C182E197E00E9404
:1043D0005D05FFC081E08170FEC0C43228F5CE319A
:1043E00008F0C1C0CB30A1F1D0F4C73009F0D3C080
:1043F0008EE18093130182E3809312018AE080931F
:10440000110184E18093100188E080930F0188E21C
:1044100080930E0188EB95E00E945D05BFC0C3311B
:1044200049F1C431C1F0B7C0CB3409F4A9C028F4B4
:10443000C93289F0C83361F0AEC0C13509F49EC0FD
:10444000C23509F499C0CE3409F0A5C06AE09EC017
:104450000E94FF1EA3C08091DA01882319F01092F8
:10446000DA019CC085EC95E00E945D0581E08093B7
:10447000DB01B1C08FE995E00E945D058DE895E014
:104480000E945D05809113011F928F938AE895E049
:104490009F938F930E94F60588E895E00E945D0542
:1044A00086E795E00E945D05809112011F928F932F
:1044B00083E795E09F938F930E94F60581E795E04F
:1044C0000E945D0582E695E00E945D0580911101E4
:1044D0001F928F938FE595E09F938F930E94F6052F
:1044E0008DE595E00E945D058CE495E00E945D05F8
:1044F000809110011F928F9389E495E09F938F9391
:104500000E94F60587E495E00E945D0582E395E050
:104510000E945D0580910F011F928F938FE295E0BD
:104520009F938F930E94F6058DE295E00E945D05B2
:1045300086E195E00E945D0580910E011F928F93A8
:1045400083E195E09F938F930E94F60581E195E0CA
:104550000E945D058DB79EB748960FB6F8949EBF32
:104560000FBE8DBF1BC0CE51EC2FF0E0E35DFE4FC0
:1045700080818093DA0112C061E003C061E006C06F
:104580006AE08091DA010E94161F08C08091DA016A
:104590000E94B91F03C086EB95E013C08091DA0139
:1045A000882369F01F928F9380EB95E09F938F9300
:1045B0000E94F6050F900F900F900F9004C08DEAA7
:1045C00095E00E945D0581E006C01092DB0180E06D
:1045D00002C080E000CFCF9108950E94F422689439
:1045E000B1110C94832308950E94682388F09F578B
:1045F00098F0B92F9927B751B0F0E1F0660F771F07
:10460000881F991F1AF0BA95C9F714C0B13091F0FC
:104610000E948223B1E008950C948223672F782FA3
:104620008827B85F39F0B93FCCF3869577956795C1
:10463000B395D9F73EF490958095709561957F4F2D
:104640008F4F9F4F0895E89409C097FB3EF49095D3
:104650008095709561957F4F8F4F9F4F9923A9F05B
:10466000F92F96E9BB279395F695879577956795EA
:10467000B795F111F8CFFAF4BB0F11F460FF1BC02E
:104680006F5F7F4F8F4F9F4F16C0882311F096E9C1
:1046900011C0772321F09EE8872F762F05C066236F
:1046A00071F096E8862F70E060E02AF09A95660F28
:1046B000771F881FDAF7880F9695879597F90895E1
:1046C00057FD9058440F551F59F05F3F71F04795C3
:1046D000880F97FB991F61F09F3F79F087950895A8
:1046E000121613061406551FF2CF4695F1DF08C0C7
:1046F000161617061806991FF1CF869571056105E4
:1047000008940895E894BB2766277727CB0197F98B
:1047100008950E949C230C940D240E94FF2338F0DE
:104720000E94062420F0952311F00C94F6230C949B
:10473000FC2311240C9483230E94602370F3959F23
:10474000C1F3950F50E0551F629FF001729FBB2788
:10475000F00DB11D639FAA27F00DB11DAA1F649F24
:104760006627B00DA11D661F829F2227B00DA11DD7
:10477000621F739FB00DA11D621F839FA00D611D5D
:10478000221F749F3327A00D611D231F849F600D7E
:10479000211D822F762F6A2F11249F5750409AF0A7
:1047A000F1F088234AF0EE0FFF1FBB1F661F771F33
:1047B000881F91505040A9F79E3F510580F00C94FE
:1047C000F6230C9483235F3FE4F3983ED4F386955D
:1047D00077956795B795F795E7959F5FC1F7FE2B9E
:1047E000880F911D9695879597F9089597F99F677A
:1047F00080E870E060E008959FEF80EC0895002469
:104800000A941616170618060906089500240A9435
:1048100012161306140605060895092E0394000CBB
:1048200011F4882352F0BB0F40F4BF2B11F460FF4A
:1048300004C06F5F7F4F8F4F9F4F0895991B79E0A2
:1048400004C0991F961708F0961B881F7A95C9F720
:104850008095089597FB072E16F4009407D077FDF6
:1048600009D00E94442407FC05D03EF49095819520
:104870009F4F0895709561957F4F0895EE0FFF1F2C
:104880000590F491E02D0994AA1BBB1B51E107C0D0
:10489000AA1FBB1FA617B70710F0A61BB70B881FD0
:1048A000991F5A95A9F780959095BC01CD0108955F
:0448B000F894FFCFAA
:1048B4002A071B08F807C40790070101B901280853
:1048C400140A321E404D3622391A03CD029702755E
:1048D400023C02AF01C801E101FA011A020102031C
:0848E4000405060708090000A5
:10680000E70000000000000004000500060007008B
:10681000080009000A000B000C000D000E000F001C
:1068200010001100120013001400150016001700CC
:10683000180019001A001B001C001D001E001F007C
:10684000200021002200230024002500260027002C
:106850002800000035002B002C002D002E002F00FA
:1068600030002A00000033003400290036003700D1
:106870003800E00000000000000000000000000000
:106880000000000000000000000000000000000008
:1068900000000000000000000000000000000000F8
:1068A00000000000000000000000000000000000E8
:1068B00000000000000000000000000000000000D8
:1068C00000000000000000000000000000000000C8
:1068D00000000000000000000000000000000000B8
:1068E0000000000000000000310000000000000077
:1068F0000000E100E300E200F1A1E500E600000095
:106900000100010001000100EA4401000100E2442D
:106910000100010001005500460054004A004B00F0
:10692000560057004700480001000100E9440100FB
:106930000100010001000100010001003A003B00DC
:106940003C003D003E003F0040004100420043004B
:10695000580001004C00390001004400450052007D
:1069600001000100010050004F0081404D004E0029
:1069700051000100010001000100010001000100BF
:1069800001000100010001000100010001000100FF
:1069900001000100010001000100010001000100EF
:1069A00001000100010001000100010001000100DF
:1069B00001000100010001000100010001000100CF
:1069C00001000100010001000100010001000100BF
:1069D00001000100010001000100010001000100AF
:1069E0000100010001000100490001000100010057
:1069F000010001000100010001000100010001008F
:00000001FF
